:1000000009C019C018C017C016C015C014C013C04D
:1000100012C011C011241FBECFE9CDBF10E0A0E671
:10002000B0E0ECE1F1E002C005900D92A037B1071D
:10003000D9F705D071C0E4CF8FEE87BB089587EA6A
:1000400091E60197F1F700C000008FEE87BBE7EA69
:10005000F1E63197F1F700C0000060E070E080E069
:1000600090E0E0E0F0E020E030E0B49919C00196C3
:100070008D32910589F46A30710581F5D901AF712E
:10008000B070A901689414F8559547951694E1F756
:10009000A417B507B1F022C08536910524F51EC01E
:1000A000E130F10529F5009789F1853091053CF1A2
:1000B000220F331F6F5F7F4F853191052CF1216037
:1000C00023C02F703070205A3F4FF901208128BB88
:1000D00060E070E0E0E0F0E020E030E04FE14A95E1
:1000E000F1F700C0C2CF82E390E042E050E010C0E0
:1000F00080E090E040E050E0E1E0F0E009C080E026
:1001000090E04FEF5FEF04C080E090E040E050E00F
:0C0110004115510519F3DCCFF894FFCF26
:10011C00000609000A0208000501040000000000A6
:00000001FF
